:100000008A0102288312031387011B30831687009D
:1000100080309400093093002830831294008C11B2
:100020008316111483160313111C17281228831228
:1000300003138C1190309300831203130C080839BA
:10004000003C0130031D0301003C031928281C2833
:10005000831203138C1140309300831203130C0896
:100060000839003C0130031D0301003C0319392805
:100070002D28F001831203138C1170089300831252
:1000800003130C080839003C0130031D0301003C38
:0A00900003194B283F28F00A3A2814
:00000001FF
